:1000000019C028C027C026C025C024C023C022C0D4
:1000100021C020C01FC01FC01DC01CC01BC01AC0F3
:1000200019C018C017C016C015C014C013C012C024
:1000300011C010C011241FBECFEFD4E0DEBFCDBF72
:1000400011E0A0E0B1E001C01D92A230B107E1F7DC
:100050002CD03FC0D5CF1F920F920FB60F92112414
:100060008F939F9388B190E1892788B9809100018F
:1000700090910101CB9754F480910001909101017E
:100080000196909301018093000108C01092010134
:100090001092000188B190E2892788B99F918F91D1
:1000A0000F900FBE0F901F9018953C9A3D9A83E8D1
:1000B0009EE19093890080938800809181008C60FC
:1000C0008093810080916F00826080936F007894AC
:0600D000FFCFF894FFCF02
:00000001FF
